:100000000C94B3060C94EB060C94EB060C94CA2BE0
:100010000C94EB060C94EB060C94EB060C94EB069C
:100020000C94EB060C94EB060C9443140C945A18A5
:100030000C94B6230C94EB060C94EB060C94EB0694
:100040000C94EB060C94EB060C94EB060C94EB066C
:100050000C94EB060C941C150C94EB060C94EB061C
:100060000C94EB060C94EB060C94EB060C94EB064C
:100070000C94EB060C94EB060C94EB060C94EB063C
:100080000C94EB060C94EB060C94EB060C94EB062C
:100090000C94EB060C94EB060C94EB060C94EB061C
:1000A0000C94EB060C94EB060C94EB062B4414001A
:1000B0001A0009001300050029210400150016008C
:1000C00017000A001A7C1D001B000600070019001B
:1000D00000000000000082522C002A282A2433004D
:1000E0001C0018000F000D00343112000C00080035
:1000F000110010001B7C3800370036000B000E008A
:10010000000000000000015228432C342B443A0028
:100110003B003C003D003E0029213F0040004100E3
:10012000420043001A7C000000000000440045002B
:10013000000000000000045200522A282A24270050
:1001400026002500240023022E002D00230022007B
:10015000210036002502380020001F001E00370055
:10016000000000000000035228432C342B441E02E0
:100170001F022002210222022921000000000000AB
:1001800062000000E100000000000000000000002C
:10019000000000000000025200522A282A242702F0
:1001A00026022502240223023500310030002F00F0
:1001B0002E002D003502310230022F022E022D02B8
:1001C000000000000000035228432C34A800AC00BB
:1001D000AB00AA00A900AE00292100000000D30056
:1001E000D100D200E100000000000000000000008B
:1001F00000000000000004520052E300DD00000097
:100200000000DC00D000CE00DE0000000000DA00BC
:10021000D9000000DF0000000000DB00CF00CD00AF
:100220000000000000000000000000002078000036
:10023000000028782778000046000000000024789D
:1002400023780000E10000000000267825780000F7
:1002500000000000000000000052E3000052000017
:100260004A004B004F005100000000000000000059
:1002700000000000000000004D004E005000520041
:1002800000000000000003522800E30000DA0281B1
:10029000FFD9F1DB20A4A62EAF00A0C000A1C800AA
:1002A000AED580A81FD300408D142000000000E0D0
:1002B00000F8C0F8E0C0FC007E180080000280F06A
:1002C00000C080F8C0E070603C383C1C003F0C0F60
:1002D0001F030701C300E08000E080F880C0F7C77B
:1002E0006F7B3930008000C000C0C2E00040383071
:1002F000381E181E0F0C0707070303212131301881
:10030000181C080C0E07060703C303014CCCC2C21D
:100310004149092B2A6A6E2424049292B1F1F1F228
:10032000E6A4A4040428282828282828636F726ECD
:100330006500209D9E9F2020BDBEBF2020DDDEDF0A
:100340002000209495962020B4B5B62020D4D5D690
:100350002000209798992020B7B8B92020D7D8D965
:100360002000209A9B9C2020BABBBC2020DADBDC3A
:100370002000202020202000A7A800AFB000C60049
:10038000CA00C800A5A600ADAE008788008F900007
:10039000C500C900C700CB008586008D8E00ABACC0
:1003A00000CFD000C600CA00C800A9AA00B1B200A0
:1003B0008B8C00CDCE00C500C900C700CB00898A58
:1003C00000919200202000532000202000432000B4
:1003D0002020004E2000000000100000000000005F
:1003E00000081C08000000000000000002000000DF
:1003F00000001000000000000000200000000000CD
:10040000000000020040E040000000000000040086
:1004100000000080C080C080000000000000E000FC
:100420008000F00000C0000000000000004000005C
:100430000000000001008100C000FE00FC00FF2061
:10044000FFF00FF000FF00000000100000000000AF
:100450009000F80000F8FF10FF84FF60FF36FF0FE8
:10046000FF3F005F000580008000C03800ECF00016
:10047000FB80FFF0FFEFFFE8FF03FF0CFF00FF0032
:10048000030000F80080FF20FFD0FFE0FEF8FFFC33
:10049000FFFF0FFF013FFF000F0001000300FE8080
:1004A000FE00C0FFC4FBFFFEFFFFFF3FFFFF07FF93
:1004B000033F000FC0000000B800FF40BEF0FFF196
:1004C000FFFEFFFFFFFF1FFF6700EF001F00000799
:1004D0000000E000FFF0FF88FFC4FFF8FFFFFFFF10
:1004E000FFFF8F7F0FFF0007FE000700000000F8EE
:1004F00000C03FF8E7FFFFFFFF1FFFFF1F3F01FFA7
:100500000B00FF000005000000E000F86080FEE343
:10051000FCFF1EFFFF23FF09FF20003F0200000F2A
:10052000004000C000FCE0FCF0FFFF7FFCFF0FFF7D
:10053000071F00010F000F0081700CF0800000E425
:10054000F8E6703FCFFF1FFF48FF0F000700004392
:1005500060F8F0FE38FE00FC0300C872CFFC000318
:100560000F01E01CE003000F00000000000000F895
:1005700006F900030007FF001012C9F0CFB47F8016
:10058000E01E0140655EE00000F00CF000807E019E
:100590008093FCC000000000000089182C46000772
:1005A00021101080091331BFFF00081AF70F000057
:1005B000444534BFB80010F008F41811FC18FB0EC5
:1005C00010F804F810201809FF0CEA1F286030F812
:1005D00020C042332100000101010101010101019C
:1005E00002020202020202020203030303030303E4
:1005F00003040404040404040505050505060606B1
:100600000606070707070708080808090909090A6D
:100610000A0A0B0B0B0C0C0C0D0D0D0E0E0E0F0F12
:100620000F101011111112121313141415151616A0
:100630001717181819191A1A1B1B1C1D1D1E1E1F0F
:100640002020212222232424252626272829292A5E
:100650002B2C2D2D2E2F3031323233343536373886
:10066000393A3B3C3D3E3F40414243444546474882
:10067000494A4C4D4E4F50515354555658595A5B58
:100680005D5E5F616264656668696B6C6D6F7072F8
:10069000737577787A7B7D7E8082838587888A8C64
:1006A0008E8F91939596989A9C9EA0A2A3A5A7A998
:1006B000ABADAFB1B3B5B7BABCBEC0C2C4C6C9CB8F
:1006C000CDCFD1D4D6D8DBDDDFE2E4E7E9EBEEF045
:1006D000F3F5F8FAFDFF00AF00AE05010902A10134
:1006E00085020901A1000509190129081500250144
:1006F0009508750181020501093009311581257FB1
:1007000095027508810609381581257F95017508C0
:100710008106050C0A38021581257F95017508812F
:1007200006C0C005010980A101850319012AB7008F
:10073000150126B700950175108100C0050C09014F
:10074000A101850419012AA002150126A002950124
:1007500075108100C005010906A101050719E029EE
:10076000E71500250195087501810295017508813D
:10077000010507190029FF150026FF0095067508D9
:10078000810005081901290595057501910295015A
:1007900075039101C009023B00020100A0FA09049F
:1007A00000000103010100092111010001224000A4
:1007B000070581030800010904010001030000008E
:1007C000092111010001227B00070582032000019D
:1007D00012010002000000081D8D3A3400010102E0
:1007E000000124034100750072006F007200610077
:1007F000200043006F0072006E0065002000720050
:1008000065007600310000001803730070006C0072
:10081000690074006B0062002E0063006F006D00C1
:100820000000040309040000000000003E5B4F5B71
:100830003E003E6B4F6B3E001C3E7C3E1C00183C55
:100840007E3C18001C577D571C001C5E7F5E1C0000
:1008500000183C180000FFE7C3E7FF000018241849
:100860000000FFE7DBE7FF0030483A060E002629CC
:1008700079292600407F05050700407F05253F00B8
:100880005A3CE73C5A007F3E1C1C0800081C1C3EDA
:100890007F0014227F2214005F5F005F5F00060963
:1008A0007F017F00006689956A006060606060007B
:1008B00094A2FFA2940008047E04080010207E2069
:1008C000100008082A1C0800081C2A0808001E102E
:1008D000101010000C1E0C1E0C0030383E3830007A
:1008E000060E3E0E060000000000000000005F0043
:1008F0000000000700070000147F147F1400242A62
:100900007F2A1200231308646200364956205000E3
:10091000000807030000001C224100000041221CC7
:1009200000002A1C7F1C2A0008083E0808000080DE
:10093000703000000808080808000000606000002F
:100940002010080402003E5149453E0000427F400D
:1009500000007249494946002141494D33001814AD
:10096000127F10002745454539003C4A494931006E
:1009700041211109070036494949360046494929AC
:100980001E000000140000000040340000000008B9
:1009900014224100141414141400004122140800FD
:1009A0000201590906003E415D594E007C121112A8
:1009B0007C007F49494936003E41414122007F4148
:1009C00041413E007F49494941007F090909010031
:1009D0003E41415173007F0808087F0000417F417C
:1009E00000002040413F01007F08142241007F4069
:1009F000404040007F021C027F007F0408107F00FF
:100A00003E4141413E007F09090906003E41512116
:100A10005E007F0919294600264949493200030131
:100A20007F0103003F4040403F001F2040201F0047
:100A30003F4038403F006314081463000304780407
:100A400003006159494D4300007F414141000204C8
:100A500008102000004141417F000402010204000F
:100A600040404040400000030708000020545478F4
:100A700040007F2844443800384444442800384427
:100A800044287F0038545454180000087E0902009E
:100A90001824241C78007F080404780000447D405A
:100AA00000002040403D00007F102844000000412D
:100AB0007F4000007C04780478007C0804047800FF
:100AC0003844444438007C1824241800182424187E
:100AD0007C007C0804040800485454542400040496
:100AE0003F4424003C4040207C001C2040201C004F
:100AF0003C4030403C004428102844004C909090EA
:100B00007C004464544C440000083641000000005E
:100B100077000000004136080000020102040200D4
:100B20003C2623263C000000000000000000C0E03E
:100B3000F0F8F81800C0F0FCFEFFFFFFFFFFFFFF1A
:100B40007E00000000F8042252E2424242E25222B9
:100B500022224282020222220204F80000F8040249
:100B600002824222428202020282422212224282F5
:100B70000204F80000F8FCDEAE1EBEBEBE1EAEDEF5
:100B8000DEDEBE7EFEFEDEDEFEFCF80000F8FCFED1
:100B9000FE7EBEDEBE7EFEFE000000000000808005
:100BA0004040202010100808101020204040808075
:100BB0008080C0C0E0E0F0F0F8F8F0F0E0E0C0C005
:100BC00080808080404020201010080810102020D5
:100BD00040408080808040C060A050B058A850B095
:100BE00060A040C0808000F8FCFEFFE000FFFFFF37
:100BF000FFFFFF80FFFFFFFFFFFFFFFFFF1F07015A
:100C000000000000001F20444A47424242474A4435
:100C1000404040404142444440201F00001F2040CB
:100C2000414040404040414041414F4848484F4189
:100C300041201F00001F3F7B75787D7D7D78757B8F
:100C40007F7F7F7F7E7D7B7B7F3F1F00001F3F7FFD
:100C50007E7F7F7F7F7F7E7F00000000000088888E
:100C60005D5D3E3E7C7CF8F87C7C3E3E5D5D888828
:100C700088885555232347478F8F4747232355554A
:100C800088888888D5D5E2E2C4C48888C4C4E2E2F2
:100C9000D5D5888888885DD56BB66DD6ADDA6DD62A
:100CA0006BB65DD5888800030F1F3F3F3F3F1F1F76
:100CB0003F3F7F7F7F3F3F1F3F7F7F7F7F7C7878F5
:100CC000381C0F0004F80000F804201F00001F204B
:100CD000FCF80000F8043F1F00001F2004F800008B
:100CE000F8FC201F00001F3FFCF80000F8FC3F1F2D
:100CF00000001F3FFE7EBEDEEEDEBE7EFEFCF80084
:100D00007E7E70777777707E7E3F1F000000000048
:100D100000000000000000000000000000000000D3
:100D20000101020204040808040402020101000097
:100D30000000010102020404080804040202010187
:100D4000000000000101030307070F0F070703035B
:100D50000101000000000101030205060D0A05065D
:100D600003020101000011241FBECFEFDAE0DEBF55
:100D7000CDBF04B603FE18C0809182069091830611
:100D8000A0918406B09185068730904BA740B04B68
:100D900059F41092820610928306109284061092E3
:100DA0008506E0E0F8E3099512E0A0E0B1E0ECE3AD
:100DB000FCE502C005900D92A239B107D9F726E0F3
:100DC000A2E9B2E001C01D92A238B207E1F70E9489
:100DD000DD230C94C82D0C94000080917104837065
:100DE00051F08460809371041092620180917004CC
:100DF000816080937004089590917104937071F0F4
:100E00008093720460937304413808F040E8409383
:100E10007404809170048160809370040895E8EDFB
:100E2000F0E080818E7F80831092E2001092DA00E1
:100E30001092E100A0EEB0E08C9181608C938081F3
:100E40008F77808319BCA7EDB0E08C918E7F8C9357
:100E500080818F7E80831092560408952091E40053
:100E60003091E50095E6A9012091EC00822F817078
:100E700020FF06C08091E80080FF06C080E0089552
:100E80002091E80022FD1AC080916304882389F034
:100E9000853089F08091EB0085FD0FC02091E40042
:100EA0003091E50042175307F9F29150E1F684E0E2
:100EB000089582E0089583E0089581E00895809187
:100EC000650487FF13C08091E80082FF06C080910F
:100ED000E8008B778093E80004C08091630481115F
:100EE000F2CF0895809163048823D9F38091E800BC
:100EF00080FFF8CF8091E8008E77ECCF982F909309
:100F0000E900242F762F50E0891731F07091EC0022
:100F10002091ED005091F00021FD07C09F5F9730B8
:100F200071F78093E90081E008953091EB003E7FF6
:100F30003093EB003091ED003D7F3093ED00309128
:100F4000EB0031603093EB007093EC002093ED00E8
:100F50005093F0002091EE0027FDE0CF80E008954F
:100F6000B0E0A0E0E6EBF7E00C94042DC8EDD0E093
:100F700088818F7E8883E7EDF0E0808181608083C7
:100F800084E082BF81E08093560488818E7F8883CD
:100F900002EE10E0F80110821092DA0081EEC82E05
:100FA000D12CF601108288818F77888388818068B0
:100FB000888388818F7D888319BC10926304109286
:100FC0006404109262041092610490EEE92EF12CF8
:100FD000F70180818B7F808388818160888342E0F4
:100FE00060E080E00E947E07F60180818E7F808332
:100FF000F801808181608083808188608083F7012F
:1010000080818E7F8083888180618883CDB7DEB7C1
:10101000E8E00C94202DFC0180916B0490916C040D
:1010200086179707A0F06115710529F49091E800E3
:101030009E779093E80090E06115710551F491114D
:1010400008C08091E80082FF34C080E00895BC01B0
:10105000F2CF809163048823C1F18530C1F1809182
:10106000E80083FD30C08091E80082FDEACF8091E6
:10107000E80080FFE1CF8091F3002091F200382F4B
:101080006115710519F02830310558F091E02830CC
:10109000310509F090E02091E8002E772093E800D8
:1010A000CBCF81918093F100615071092F5F3F4F49
:1010B000E7CF80916304882341F0853041F080912F
:1010C000E80083FFBECF81E0089582E0089583E0C9
:1010D00008958091580408952FB7F89460915204B0
:1010E0007091530480915404909155042FBF08953A
:1010F0009C01FC0132969FEF80E04191461751F030
:101100009F3F19F4411101C0982F8F5F8630A9F7D6
:101110009F3F09F40895290F311D97FD3A95F90174
:1011200062830895A3E0B0E0E8E9F8E00C940A2DAA
:1011300020914F043091500428173907A1F0909363
:10114000500480934F04E0914D04F0914E04309789
:1011500051F024E029839B838A830680F781E02D68
:10116000CE01019609952396E2E00C94262DA3E08A
:10117000B0E0EDEBF8E00C940A2D20914B04309197
:101180004C0428173907A1F090934C0480934B042A
:10119000E0914D04F0914E04309751F023E0298303
:1011A0009B838A830680F781E02DCE010196099505
:1011B0002396E2E00C94262DCF93DF9320918006B6
:1011C000309181062A573440A901460F571F4130FC
:1011D000524020F060E072E0621B730B4091780493
:1011E00050917904FC01C901620F731FC1E0D0E086
:1011F0008617970738F05093790440937804DF916D
:10120000CF9108952491DC01A658BB4F3C91321731
:1012100081F02C939C01A5E036952795AA95E1F7DE
:10122000DE0102C0AA0FBB1F2A95E2F79D014A2BDF
:10123000532B01963196DCCFFC01680F791F8FEF9D
:1012400091E32191822728E030E087FF09C0880FD1
:10125000892721503109C9F7E617F70791F7089553
:10126000880FF7CFFA01811101C0FB01099508959C
:101270007C990FC08B3191057CF04B97FC01EE0FF0
:10128000FF1FE80FF91FED55FC4F61834083228358
:1012900003C08B31910594F30895E1E7F4E02481D4
:1012A00030E1231B08F420E02483809170048160E6
:1012B000809370040895E1E7F4E0248130E1230F86
:1012C00008F42FEF24838091700481608093700470
:1012D0000895E1E7F4E0438120E1421B08F440E097
:1012E0008181628190E00E94FC060895E1E7F4E0CC
:1012F000438120E1420F08F44FEF8181628190E049
:101300000E94FC060895E1E7F4E0628120E1621B9F
:1013100008F460E08181438190E00E94FC0608951A
:10132000E1E7F4E0628120E1620F08F46FEF818170
:10133000438190E00E94FC060895E1E7F4E081819A
:10134000438162818850990B0E94FC060895E1E771
:10135000F4E0818190E04381628108960E94FC065E
:1013600008958091710486958695815009F481E0F5
:101370000E94ED06089581E00E94ED060895FF9217
:101380000F931F93CF93DF93182F062FF42ED0E0E7
:10139000C0E02F2D402F612FCE010E9438092196E9
:1013A000C633D105B1F7CDB7DEB7E5E00C94232DF8
:1013B0008091900380FD16C081FD16C082FD16C08D
:1013C00080918F038823A1F0883280F428E0829FE7
:1013D000C001112468E270E00E943D2D862F672B2A
:1013E00039F0089582E0089584E0089588E0089532
:1013F00081E008958091900380FD14C081FD14C0A8
:1014000082FD16C080918E03882381F08E3180F496
:1014100020E5829FC00111246EE170E00E943D2D05
:10142000862F089584E1089588E2089588E008955C
:1014300080E5089580E00895F894E82FE295EF7034
:10144000F0E031A1282F2F7081E090E001C0880FDB
:101450002A95EAF7982F9095932391A392A1892B2F
:1014600082A37894089590914A0392FF06C0282F92
:1014700028712830F9F4877F846093FF06C0282FF5
:1014800028712831F1F4877E846120914B0320FF7D
:1014900006C0382F38713830D9F4877F816021FF3A
:1014A00006C0282F28712831D1F4877E816194FDF0
:1014B000877E0895282F24712430F9F68B7F886069
:1014C000DCCF282F2471243101F78B7E8861DDCF9A
:1014D000382F3171313019F78E7F8860E0CF282F97
:1014E0002171213121F78E7E8861E1CF823891050B
:1014F000B9F1B0F48133910509F47DC048F4893223
:10150000910509F46DC08A32910509F47BC00895F4
:101510008533910509F45FC08933910509F1089578
:10152000833E9105D9F138F4803E910529F1823E40
:10153000910579F10895863E9105D9F1873E91058F
:1015400009F43EC0843E910541F520914B0321FFF3
:1015500024C080914A0384FD19C087EE90E008956D
:1015600020914A03237009F05AC020914B0323FFB6
:1015700014C089E290E0089520914A0320FD38C00C
:1015800030914B0330FF09C024FF43C090E080E05E
:10159000089520914A0322FDF7CF089520914A0330
:1015A00022FD3AC030914B0330FD39C024FFF5CF06
:1015B000EDCF20914A0323FFF0CF24FDE7CFCDCF1D
:1015C00020914A0323FD2EC030914B0331FFEECF13
:1015D00084EE90E0089520914A0325FFDECFC9CF25
:1015E00020914A0325FD21C020914B0323FFD5CF35
:1015F00089E390E0D2CF20914A0326FFCECF8AE242
:1016000090E0089520914A0326FFC7CF81E390E040
:10161000089583EE90E0089582EE90E0089580EEC4
:1016200090E0089586EE90E0089585E390E00895B7
:10163000972F7830B8F46630A8F48530B0F470E0B5
:1016400026E0929F600D711D1124FB0190E3899F9C
:10165000E00DF11D1124EE0FFF1FE455FF4F8591A2
:101660009491089580E090E0089581E0FCCF1F936D
:10167000CF93DF930E94760AEC01C11580E5D8076D
:10168000F0F5C11580E4D80708F09CC0C03ED10534
:1016900020F5CD3CD10508F082C0C83AD10578F4D8
:1016A000C53AD10508F073C0C130D10519F12097B2
:1016B00009F1C430D105F0F4D0E0C0E01BC0C33C58
:1016C000D105D0F7C85AD0E0CC0FDD1FC159DE4F8D
:1016D0000990D881C02DD4640DC0C11580E2D8070F
:1016E00008F0D1C0C11581E0D80708F05AC0C83E43
:1016F000D10510F7CE01DF91CF911F910895C0362B
:1017000082E5D80718F5C03482E5D80708F06BC029
:10171000C03282E5D80708F05FC0C11582E5D8075E
:1017200008F497C02C2F2695269580E2289F9001DB
:1017300011248C2F8370C1E0D0E002C0CC0FDD1FDC
:101740008A95E2F7C22BD32BDD68D4CFC03A82E56D
:10175000D80760F4C03882E5D80708F459C0CF71C3
:10176000D0E0DC2FCC27C46FD06AC4CFC03C82E568
:10177000D80708F462C0C03E82E5D80708F09CCFC5
:10178000DC2FCC27CC27DF71C06FD06AB3CFC55A0E
:10179000D0E0C459DE4FC881D0E0D064ABCFD06573
:1017A000A9CF8D2F0E94330A182FCE0199270E94AE
:1017B000760AC12FD0E0DC2FCC27CC27DF71C82BD5
:1017C000D92B98CFCE0199270E94760ACC27DF70BB
:1017D000C82BD92BD06A8ECFCF71D0E0DC2FCC278D
:1017E000C16FD06A87CF2C2F26952695277080E26F
:1017F000289F900111248C2F8370C1E0D0E002C09B
:10180000CC0FDD1F8A95E2F7C22BD32BDC6872CF99
:101810002C2F26952695277080E2289F9001112471
:101820008C2F8370C1E0D0E002C0CC0FDD1F8A9501
:10183000E2F7C22BD32BDA685DCF8C2F8F710E9419
:10184000330AC82FD0E0DC2FCC27CC27DF71D06241
:1018500051CF8C2F8F710E94330A55E0D695C795D2
:101860005A95E1F7CF70D0E0DC2FCC27282F30E05D
:1018700084FF05C044E0220F331F4A95E1F7C22BD5
:10188000D32BD06937CF8D2F8F710E94330A182F39
:10189000CE0199270E94760AC12FD0E0DC2FCC27F9
:1018A000CC27DF71C82BD92BD2CF0E946C080895AA
:1018B000809168038111109268030895809590913A
:1018C000670398239093670308952091EC02909109
:1018D000BB0256E0291302C080E0089530E0529F19
:1018E000F001539FF00D1124E454FD4F71817613E4
:1018F00006C07081781303C07281741304C02F5F17
:101900003F4F2770E7CF81E008958091EC029091DE
:10191000BB02981301C008958F5F8770FACFB0E0C3
:10192000A0E0E5E9FCE00C94032D7C010091650347
:10193000109166038091F7029091F802082B192B01
:10194000CFE0D0E0CC24C394D12CBC2EC6010C2E09
:1019500002C0880F991F0A94E2F780239123892BF4
:1019600049F4219790F7B12C8B2DCDB7DEB7E9E084
:101970000C941F2DB7018C2F0E94180B0E94370B5F
:10198000019779F3F1CFCF93DF93EC010E948F0C95
:10199000BE010E94180B0E94370BDF91CF91089572
:1019A000983078F5863068F5E82FF0E086E0989F6B
:1019B000E00DF11D11249E2F977083E0F695E795B9
:1019C0008A95E1F7EE0FFF1FEE0FFF1FE356FD4F65
:1019D00050E040E080E0219130E0092E02C03695D1
:1019E00027950A94E2F721703327042E01C0220FB5
:1019F0000A94EAF7822B4F5F5F4F4430510559F745
:101A0000089580E00895983098F5863088F5E82F9D
:101A1000F0E086E0989FE00DF11D11248E2F877075
:101A200041E001C0440F8A95EAF783E0F695E79517
:101A30008A95E1F7EE0FFF1FEE0FFF1FE356FD4FF4
:101A400030E020E070E05191DF011197CB01022ED0
:101A500002C0969587950A94E2F781708195852753
:101A6000842385278C932F5F3F4F2430310559F70E
:101A700008959093660380936503089521E030E014
:101A800002C0220F331F8A95E2F72095309580918E
:101A9000650390916603822393230E94390D089574
:101AA0009091ED02809589238093ED02282F277075
:101AB00091F4282F082E000C330B9217130659F0BF
:101AC00090914B0392FF07C08595859585950E945F
:101AD0003E0D1092ED02089521E030E002C0220F89
:101AE000331F8A95E2F78091650390916603822BFC
:101AF000932B0E94390D08959093F8028093F7027A
:101B00000895FC0183819481892B29F08081918142
:101B100089238F3F51F480E00895843FE1F717C097
:101B2000883EA8F0813FB9F712C0808191810E9460
:101B3000C30C92959F70963099F358F4925F9F7002
:101B4000923048F7803F19F040F7883E20F781E057
:101B500008959A5FF4CFCF93DF93C0918006D09120
:101B600081068A30C1F420917704CE018A579440CF
:101B7000622F70E00E94E62C281B822F66E00E94F4
:101B8000312DC82FC15018F4DF91CF91089580E214
:101B90000E94AB0DF7CF8D30E9F4CA57D4402091A5
:101BA0007704622F70E0CE010E94E62C281B822F62
:101BB0009E01280F311D2115324018F080E0D0E041
:101BC000C0E0C80FD11DC658DB4FD0938106C0932B
:101BD0008006DACF96E0FE01AAE7B6E001900D920A
:101BE0009A95E1F7803E08F458C086E0FE01119214
:101BF0008A95E9F7C0918006D091810646E050E0D1
:101C0000BE018AE796E00E94602D9E012A5734406B
:101C1000892B41F1C90145E0969587954A95E1F7F1
:101C200041E050E0BA0102C0660F771F8A95E2F7E3
:101C3000CB016091780470917904862B972BB901C0
:101C40006B5F7F4FE5E076956795EA95E1F702C017
:101C5000440F551F6A95E2F7842B952B90937904D6
:101C6000809378042A5F3F4F40917704642F70E09F
:101C7000C9010E94E62C481B463010F4240F311D88
:101C8000211572E0370710F030E020E026583B4F76
:101C9000309381062093800677CFF6E08F9FB001C6
:101CA00011246A5D774F46E050E0CE010E94572D27
:101CB000A1CFCF93DF93EC01FE018491811103C08A
:101CC000DF91CF9108950E94AB0D2196F5CF8091C1
:101CD00067039091F602892B809394029091680398
:101CE000992391F0892B8093940220E086E992E079
:101CF000FC013191CF0131112F5FF2E08C399F0748
:101D0000B9F721110E94580C48E050E06EEE72E0E5
:101D100084E992E00E94602D892BA9F088E0E4E933
:101D2000F2E0AEEEB2E001900D928A95E1F7E0911B
:101D30004D04F0914E04309731F00280F381E02D94
:101D400084E992E009950895882321F00E945E0CB1
:101D50000E94670E0895882339F090916703982BAD
:101D6000909367030E94670E0895B0E0A0E0EBEB4C
:101D7000FEE00C94042D6C017B0164E670E088E7C2
:101D80000E94442AEC0197FD12C010E000E0F60129
:101D9000E00FF11F849164E670E00E94B02AEC012C
:101DA000892B29F40F5F1F4F0E151F0581F70E9425
:101DB000262BCE01CDB7DEB7E8E00C94202D809124
:101DC000490490914A04911103C091E08927089534
:101DD000882369F062E070E088ED96E00E94B50E1D
:101DE000892B19F08091490408951092490480913B
:101DF0004904EBCFCF93C091490480914A048823D2
:101E0000D1F00E946C08605A75418F4F9F4F6093CC
:101E10004504709346048093470490934804C1118D
:101E200008C062E070E086ED96E00E94B50E892B56
:101E300029F0C09149048C2FCF91089581E08093BF
:101E40004904F7CF0F931F93CF93DF938B01EA01E0
:101E500090916304943061F58093E9008FEF909145
:101E6000E800815095FD06C095ED9A95F1F70000C8
:101E70008111F5CF8091E80085FF1AC00E942E07DE
:101E8000811111C08091E80085FD06C08091E800B5
:101E90008E778093E800F2CFF80181918F018093D3
:101EA000F100219779F78091E8008E778093E80020
:101EB000DF91CF911F910F91089543E050E0BC0155
:101EC00082E00E94220F089546E050E0BC0182E0CB
:101ED0000E94220F0895CF93DF93EC0148E050E079
:101EE000BC0181E00E94220F88E0FE01A9E5B4E078
:101EF00001900D928A95E1F7DF91CF91089581E0ED
:101F00008093E00080E28093D8001092C9008FE1B6
:101F10009EE40197F1F700C0000087E090EBDC0140
:101F20008093820690938306A0938406B0938506DF
:101F300088E19CE00FB6F894A895809360000FBEEE
:101F400090936000FFCF539A3BB1377F2BB128604D
:101F50004FB7F89483EA93E0FC015191CF0168E018
:101F60002BB9000000C057FF3BB9550F000000C05F
:101F700000C000C03BB900C06A9591F7F4E0853419
:101F80009F0751F74FBF8FE594E00197F1F700C02D
:101F900000000895B0E0A0E0E0EDFFE00C94022D19
:101FA0007C015B016A018091390301E010E08A3015
:101FB00010F40AE010E0C1E0D0E0B501C701F6017D
:101FC0000995811104C021960C171D072CF4CDB77B
:101FD000DEB7EAE00C941E2DCC9F9001CD9F300D12
:101FE000300D112490E080E045E34A95F1F70000C0
:101FF000019682179307C1F7E0CF80910503811105
:1020000010C08091D80080618093D8008AE18A95C1
:10201000F1F700C08091D90080FF0AC081E0809371
:10202000050381E090910503913009F080E0089567
:1020300082E0809305030E940F0710926304F1CFA2
:102040000E94FD0F882359F0E0914D04F0914E0459
:10205000309729F00190F081E02D0995089580E0F6
:1020600008950F931F930E94FD0F882329F00E946B
:102070006C081F910F9108950E946C0800913A031B
:1020800010913B0320913C0330913D03600F711F81
:10209000821F931FEECFB0E0A0E0E1E5F0E10C94E9
:1020A000002D0E94311060939B0370939C038093DA
:1020B0009D0390939E0330917104D32FD37019F038
:1020C000D32FD695D695209162012130D9F02223C5
:1020D00059F0223009F413C1233009F419C1CDB7E6
:1020E000DEB7ECE00C941C2D10925E0160939F0310
:1020F0007093A0038093A1039093A20381E0809347
:102100006201EDCF90915D0181E0D9130BC0832F67
:10211000837020915C0130E091E08217130609F48E
:1021200090E0892F81708093600180917604909176
:102130005F01981739F080935F0140E060E080E034
:102140000E94BF09DD2321F0D13061F080E03AC068
:10215000809160018823B1F140E060E080E00E945E
:10216000BF09F4CF90905E018BE0989E902C1124D3
:102170001BE0190D173308F016E37C9B03C01C31DC
:1021800008F01BE17C9906C02BE1C22E9C1410F4D0
:102190009BE1992E40917204D0907304E0917404F5
:1021A000F0E0EA52FA4FD1101FC0F4900F2DCF2D5E
:1021B000C92CD12CC11608F48CC081E07C9B9BC03B
:1021C0001B3120F690915E019F5F90935E0181111B
:1021D00086CF82E0809362018091600181117FCF80
:1021E000D1117DCF83E08BCFED2CF12CC4918C2EBF
:1021F000EC2FF0E026E0429FC00111242FEF30E0E9
:10220000B9010E94E62CA42FB0E0AA0FBB1F45E540
:10221000469FC001479F900D1124AD01481B590BEB
:10222000A42FAA0FA40FC9018E199F098E9FA00188
:102230008F9F500D9E9F500D1124052FDA9EC001D7
:102240001124892F99276901C81AD90ACE9E5001F5
:10225000CF9EB00CDE9EB00C11246901CA1AD108C1
:10226000CE9CD001CF9CB00DDE9CB00D1124AB2FC5
:10227000BB272A1B3B0B2E9FC0012F9F900D3E9F1B
:10228000900D1124F92E62307105A1F050F4611502
:10229000710509F48DCF6130710581F0F52E0B2D9C
:1022A00087CF6430710569F080F06630710509F4FC
:1022B0007FCFF4CFFC2EC52F092F7ACFFC2ECB2D4C
:1022C00077CFF52E0C2FC92F73CFC52F082DFB2CE0
:1022D0006FCFF601E55AFD4F808190915F01892310
:1022E00031F0202F4F2D6C2FC6010E9438092FEF9F
:1022F000C21AD20A5FCF163308F464CF27CFD09327
:102300005D01832F837080935C010E94A30F6ACFCD
:1023100080917004882351F046E050E06CE170E059
:1023200081E794E00E94942D10927004C0909F0366
:10233000D090A003E090A103F090A2030E94FD0FB3
:102340008823C1F02FB7F894609152047091530420
:1023500080915404909155042FBF6C197D098E090A
:102360009F09603171058105910508F4B8CE10927E
:102370006201B5CE0E943110F0CFE1E7F4E085E0D4
:1023800080838091630190916401A09165018183B4
:102390009283A3838FE784838FEF858346E050E0A9
:1023A0006CE170E0CF010E94942D109270040895AA
:1023B00090914B0392FB222720F9281779F080FB9C
:1023C00092F990934B0360914A0370914B0384E020
:1023D00090E00E94C22D82E00E94500D0895A4E07A
:1023E000B0E0E5EFF1E10C94092D40912D035091FF
:1023F0002E0360912F03709130032FB7F8948091D2
:10240000520490915304A0915404B09155042FBFED
:10241000841B950BA60BB70B11E084369105A10523
:10242000B10570F10E9431106E5F7F4F8F4F9F4F4B
:1024300069837A838B839C838091290190912A01FF
:102440008A5E9C4F4091280150E04530510510F0C4
:1024500044E050E0BE016F5F7F4F0E946D2D85E02C
:1024600090E00E94702C182F882351F00E946C0875
:1024700060932D0370932E0380932F03909330036A
:10248000812F2496E3E00C94252D4F925F926F925A
:102490007F928F929F92AF92BF92EF92FF920F9393
:1024A0001F93CF93DF937B01FB01408051806280BB
:1024B00073809FB7F8948090520490905304A0903A
:1024C0005404B09055049FBF84189508A608B70817
:1024D000F4E68F169104A104B10418F4C1E044237A
:1024E00029F1C82F880FDD0BFE0183E0EE0FFF1FDF
:1024F0008A95E1F7E050FF4F818192818A5E9C4F7F
:10250000408150E00417150708F4A801B9010E94A2
:102510006D2DCE010E94702CC82F882339F00E94A7
:102520006C08F70160837183828393838C2FDF9122
:10253000CF911F910F91FF90EF90BF90AF909F9020
:102540008F907F906F905F904F900895A1E0B0E0E2
:10255000ECEAF2E10C94082D8091490489832091E2
:102560002C0390E041E02817190609F440E001E04F
:1025700010E09E012F5F3F4F65E373E087E00E940C
:1025800045122196E4E00C94242DA7E0B0E0EBEC9A
:10259000F2E10C94082D86E0E1E7F4E0DE0111960B
:1025A00001900D928A95E1F71F8247E050E065E2C5
:1025B00073E0CE0101960E94602D41E0892B09F461
:1025C00040E007E010E09E012F5F3F4F61E373E0C2
:1025D00086E00E9445122796E4E00C94242D0F9388
:1025E0001F93CF93DF93EC0144E050E06BE173E085
:1025F0000E94602D41E0892B09F440E004E010E0E6
:102600009E016EE073E082E00E944512DF91CF915F
:102610001F910F9108954F925F927F928F929F9298
:10262000AF92BF92CF92DF92EF92FF920F931F93E0
:10263000CF93DF930F92CDB7DEB7C62E4A01590173
:10264000482E880F5508C2010E94702C782E8823CE
:1026500009F480C0C20133E0880F991F3A95E1F771
:10266000FC01E050FF4F438150E04115510511F04E
:1026700041E050E080509F4FFC01648175816A5EAB
:102680007C4FCE0101960E946D2DF4014081518155
:10269000628173812FB7F894809152049091530412
:1026A000A0915404B09155042FBF841B950BA60B29
:1026B000B70B84369105A105B10540F4B701C801F7
:1026C0000E941C099981891709F444C00C2C000C44
:1026D000DD08C6010E94702C782E811113C0712C68
:1026E000872D0F90DF91CF911F910F91FF90EF9069
:1026F000DF90CF90BF90AF909F908F907F905F9032
:102700004F900895C60123E0880F991F2A95E1F79D
:10271000FC01E050FF4F438150E0E416F50608F459
:10272000A70180509F4FFC01648175816A5E7C4FD8
:10273000C5010E946D2DB701C8010E941C09998135
:102740008913CDCF0E946C08F4016083718382836A
:102750009383C6CFA701B801C5010E946D2DC0CFDC
:10276000A4E0B0E0E6EBF3E10C94042D6B0184E00F
:10277000E82EF12C07E113E09E012F5F3F4F4AE066
:1027800053E061E080E00E940B13882361F04981EF
:102790005A816B817C8140930603509307036093B9
:1027A0000803709309034091060350910703609159
:1027B000080370910903F601408351836283738398
:1027C0002496E8E00C94202D67EE7EEF90E080E008
:1027D0000E94C22D60E082E090E00E94A42D60E0A3
:1027E00083E090E00E94A42D1092F8021092F7026C
:1027F00060E074E184E090E00E94C22D60E086E039
:1028000090E00E94A42D6FEF87E090E00E94A42D3D
:1028100040E050E0BA0188E090E00E94B62D60E010
:102820008DE090E00E94A42D40E050E0BA0188E1E4
:1028300090E00E94B62D60E087E190E00E94A42D18
:1028400040E050E0BA018CE190E00E94B62D70E0CB
:1028500060E080E290E00E94C22D40E050E0BA01CA
:1028600088E190E00E94B62D40E050E0BA018FE090
:1028700090E00E94B62D40E050E0BA0183E190E084
:102880000E94B62D08951F920F920FB60F92112439
:102890002F933F934F935F936F937F938F939F9368
:1028A000AF93BF93EF93FF938091E10082FF09C044
:1028B0008091E20082FF05C08091E1008B7F8093D0
:1028C000E1008091DA0080FF24C08091D80080FF71
:1028D00020C08091DA008E7F8093DA008091D90049
:1028E00080FF9DC080E189BD82E189BD09B400FE01
:1028F000FDCF81E08093630480915604811109C06B
:102900000E940F070E94B0078091E20084608093CC
:10291000E2008091E10080FF17C08091E20080FF1B
:1029200013C08091E2008E7F8093E2008091E200EC
:1029300080618093E2008091D80080628093D8000B
:1029400019BC85E0809363048091E10084FF2BC073
:102950008091E20084FF27C080E189BD82E189BDCA
:1029600089B5982F917080FFFBCF8091D8008F7D23
:102970008093D8008091E1008F7E8093E100809168
:10298000E2008F7E8093E2008091E200816080937C
:10299000E20080916404882309F447C084E08093B6
:1029A0006304809163048091E10083FF27C08091DC
:1029B000E20083FF23C08091E100877F8093E100E4
:1029C00082E080936304109264048091E1008E7F22
:1029D0008093E1008091E2008E7F8093E2008091FD
:1029E000E20080618093E20042E060E080E00E94CB
:1029F0007E078091F00088608093F000FF91EF9156
:102A0000BF91AF919F918F917F916F915F914F9106
:102A10003F912F910F900FBE0F901F90189519BCEA
:102A2000109263041092560474CF8091E30087FDE6
:102A300093E090936304B5CF78941F921FB61F92D2
:102A400011248F939F93AF93BF93809152049091E1
:102A50005304A0915404B09155040196A11DB11DD9
:102A60008093520490935304A0935404B09355045C
:102A7000BF91AF919F918F911F901FBE1F9018958E
:102A80009C014FB7F8948091520490915304A09107
:102A90005404B09155044FBF821B930B08952FB778
:102AA000F8948091520490915304A0915404B091F1
:102AB00055042FBF08950E944F159C0190919703D4
:102AC00080919803982B21F03093940320939303E3
:102AD0009091990380919A03982B21F0309392035F
:102AE00020939103E0914D04F0914E04309749F00A
:102AF00082E0809395030480F581E02D85E993E0E1
:102B000009950895CF9310926703C6E0E6E9F2E0D5
:102B1000DF018C2F1D928A95E9F790E080E00E94FA
:102B2000B70890E080E00E9492081092F6020E949E
:102B3000670EE5E9F3E0DF011D92CA95E9F710920F
:102B40008E0310928F03109290030E945B15CF9119
:102B50000895AAE2B0E0EFEAF5E10C94092D85E6CC
:102B600094E02091F100FC012193CF01F4E08D3637
:102B70009F07B9F780916604833009F470C0B8F4F8
:102B8000813009F447C0823009F4B1C08091E80077
:102B900083FF7EC280916504909166049A3008F0AC
:102BA00077C2E92FF0E0E653F24D0C94512D8A30B4
:102BB00009F48CC08B3009F46FC0893039F78091EB
:102BC0006504813219F78091690490916A04029733
:102BD000E8F68091E800877F8093E8008091E80024
:102BE00082FF38C09091F3008091F200029731F497
:102BF0008091F100813011F0863021F48091F10054
:102C0000809358048091E8008B778093E8000E94BD
:102C10005F07BCCF80916504813A09F0B7CF8091FE
:102C2000E800877F8093E8008091690490916A04AE
:102C3000892B61F468E089E594E070E00E940B085C
:102C40008091E8008B778093E800A0CF60E090E06F
:102C500080E0F3CF809163048111C0CF97CF809142
:102C60006504813A09F092CF8091690490916A04D9
:102C7000892B09F08BCF8091E800877F8093E80053
:102C80008091E80080FFFCCF809161018093F1008A
:102C90008091E8008E77B9CF80916504813209F088
:102CA00075CF8091690490916A04892B09F06ECFE9
:102CB0008091E800877F8093E8000E945F07809101
:102CC0006704809361010E94821560CF8091650442
:102CD000813209F05BCF8091E800877F8093E80024
:102CE0000E945F0780916804809357044FCF8091C2
:102CF0006504813A09F04ACF8091E800877F80938C
:102D0000E8008091E80080FFFCCF80915704BECF9F
:102D1000803899F0823809F0BBC1809169048F70C6
:102D2000873008F0B5C18093E9008091EB0085FB06
:102D3000882780F91092E90006C080916104909183
:102D40006204911182609091E800977F9093E8006F
:102D50008093F1001092F1008091E8008E7794C189
:102D6000882309F482C1823009F092C180916704FE
:102D7000811185C1809169048F702FEF280F263053
:102D800008F086C18093E9002091EB0020FF77C115
:102D9000933031F48091EB0080628093EB006FC13F
:102DA0009091EB0090619093EB0021E030E001C046
:102DB000220F8A95EAF72093EA001092EA008091A8
:102DC000EB008860EACF811163C1109167041F771F
:102DD0008091E3008078812B8093E3008091E8006C
:102DE000877F8093E8000E945F078091E80080FF62
:102DF000FCCF8091E30080688093E30082E01111B2
:102E000083E08093630444C18058823008F040C15D
:102E100080916704909168048C3D23E09207A1F5AE
:102E200083E08A838AE289834FB7F894DE011396A0
:102E300020E03EE051E2E32FF0E050935700E491B0
:102E400020FF03C0E295EF703F5FEF708E2F90E0A0
:102E5000EA30C0F0C7968D939D932F5F243159F7C8
:102E60004FBF8091E800877F8093E8006AE270E0BE
:102E7000CE0101960E940B088091E8008B77809329
:102E8000E80006C1C096E7CF4091690450916A04FA
:102E9000292F33272330310509F444C078F5213038
:102EA000310509F46FC08BE390E0E5E9F7E02230EB
:102EB000310509F0EDC02091E800277F2093E8005C
:102EC00020916B0430916C048217930708F49C01E5
:102ED00040E02115310509F064C0411162C08091C4
:102EE000E80082FDC9CF80916304882329F28530F0
:102EF00019F28091E80083FFF2CFBECF2132310575
:102F0000A9F12232310509F0C3C04115510509F478
:102F100043C04130510509F0BBC08BE790E0EAEDBA
:102F2000F6E0C9CF992781309105C1F0009759F09B
:102F3000029709F0ADC0E2EEF7E0E4918E2F90E049
:102F4000E2EEF7E007C0E2E2F8E0E4918E2F90E0D5
:102F5000E2E2F8E0009709F49BC0ADCFE8E0F8E0CA
:102F6000E4918E2F90E0E8E0F8E0F4CF41155105B0
:102F700071F04130510509F08BC089E090E0E0EC40
:102F8000F7E099CF82E190E0E0EDF7E094CF89E0BF
:102F900090E0E7EAF7E08FCF80E490E0E5E5F7E046
:102FA0008ACF80916304882309F466CF853009F4C1
:102FB00063CF8091E80083FD5FCF8091E80082FDC0
:102FC0008ECF8091E80080FF84CF9091F3008091B4
:102FD000F2002115310519F08830910550F041E0DB
:102FE000089709F040E08091E8008E778093E80030
:102FF00070CF44914093F1003196215031090196F0
:10300000E8CF803809F044C08091E800877F809342
:10301000E800809164048093F1009ECE811138C055
:10302000109167041230A0F58091E800877F8093AB
:10303000E800109364040E945F07112311F084E0FC
:1030400005C08091E30087FDFACF81E0809363049F
:1030500042E061EC81E00E947E0742E261EC82E0A6
:103060000E947E078091630413C0809167048130C1
:1030700079F481E0933009F080E08093620410924B
:10308000E9008091E800877F8093E8000E945F0755
:103090008091E80083FF0AC08091E800877F8093D9
:1030A000E8008091EB0080628093EB00AA96E3E059
:1030B0000C94252D1F920F920FB60F9211242F936F
:1030C0003F934F935F936F937F938F939F93AF93B0
:1030D000BF93CF93DF93EF93FF93D091E900DF701D
:1030E0008091EC00C82FC17080FDC0E81092E9000B
:1030F0008091F000877F8093F00078940E94A9155A
:103100001092E9008091F00088608093F000CD2B50
:10311000CF70C093E900FF91EF91DF91CF91BF9104
:10312000AF919F918F917F916F915F914F913F915F
:103130002F910F900FBE0F901F9018950E9482152F
:103140002FEF84E39CE0215080409040E1F700C0E5
:10315000000088E19CE00FB6F894A8958093600089
:103160000FBE90936000FFCF662309F45DC08D3CD5
:1031700041F40E94FA098195809398030E945B159F
:1031800008958E3C19F40E94FA09F6CF8F3C31F471
:103190000E94FA09819580939703F0CF803D19F43E
:1031A0000E94FA09F8CF893D29F40E94D80980933A
:1031B0009903E4CF8A3D21F40E94D8098195F7CF85
:1031C0008B3D31F40E94D809819580939A03D6CF24
:1031D0008C3D19F40E94D809F8CF9FE2980F9830DF
:1031E00070F4815D990B21E030E001C0220F8A95D7
:1031F000EAF780919603822B80939603BFCF8D3D93
:1032000031F480919003816080939003B7CF8E3D1D
:1032100021F4809190038260F7CF8F3D09F0AECF0B
:10322000809190038460F0CF409197038D3C59F4D6
:103230008091980387FF0DC01092980341110BC035
:1032400010928E0308C08E3C81F48091980318166A
:103250009CF3442381F08091990390919A03892BE8
:1032600009F08CCF10928F0389CF8F3C49F447FF30
:10327000F0CF10929703809198038111ECCFE0CFAB
:10328000803D19F41416ACF3E4CF90919903893D75
:1032900029F41916F4F610929903DBCF8A3D19F43C
:1032A00097FFD7CFF8CF90919A038B3D29F497FFE2
:1032B000D0CF10929A03CDCF8C3D19F41916CCF3D0
:1032C000C8CF9FE2980F983090F4815D990B21E070
:1032D00030E0B90102C0660F771F8A95E2F7CB0193
:1032E000809590919603892380939603B2CF8D3D6C
:1032F00031F4809190038E7F80939003AACF8E3D0E
:1033000021F4809190038D7FF7CF8F3D09F0A1CFFD
:10331000809190038B7FF0CF8823D1F19CEF980FA1
:10332000913A78F4E6E9F2E09191891303C0DF0164
:1033300011971C9292E0EC39F907B1F70E94670EE1
:10334000089590E2980F983050F4877091E001C092
:10335000990F8A95EAF7892F0E945E0CEFCF9BE5C3
:10336000980F933028F490E080E00E94B708089509
:1033700098E5980F9B3128F490E080E00E94920835
:10338000089593E3980F933118F460E00E94B41805
:103390000895CF93C82F8823B1F08CEF8C0F813A1A
:1033A00000F5E6E9F2E08CE992E0DF012D91C21729
:1033B00061F08A179B07D1F76C2F84E992E00E9495
:1033C00078080E94670ECF9108952191C21303C01F
:1033D000DF0111971C928E179F07B9F70E94670EA5
:1033E000EBCF80E28C0F883068F4C77021E030E0CA
:1033F00001C0220FCA95EAF780916703822B809360
:103400006703DFCFEBE5EC0FE33040F4F0E0E45985
:10341000FE4F808190E00E94B708D5CFE8E5EC0F21
:10342000EB3150F4F0E0EE0FFF1FE159FE4F8081C9
:1034300091810E949208C7CF83E38C0F833118F6E5
:1034400061E08C2F0E94B418BECF1F93CF93DF93FF
:10345000182FEB010E94C919209739F4812F0E947F
:103460008C19DF91CF911F9108958FE99FE001970B
:10347000F1F700C000002197EFCF0F931F93CF9378
:10348000DF93C62FD42F022FFC0182818823A9F05D
:1034900060936F040E944F1590936E0480936D04A7
:1034A000C77081E001C0880FCA95EAF70E94AB0E91
:1034B000DF91CF911F910F91089580916F04681350
:1034C00034C080916D0490916E040E944015883C38
:1034D000910558F510E21D0FCD17B9F080E28C0F61
:1034E000883040F4C77081E001C0880FCA95EAF7C0
:1034F0000E94A40E183048F481E09D2F977001C0FF
:10350000880F9A95EAF70E94AB0E70E060E0802F7A
:103510000E94251A183060F6D77081E001C0880F2C
:10352000DA95EAF70E94A40EC3CFC77081E001C00C
:10353000880FCA95EAF7F6CF81110CC070E06623B8
:1035400031F060E089EA0E94251A81E0089560E088
:103550008AEAF9CF8130C9F770E0662319F060E09C
:103560008EE4F1CF60E08BE4EECFA1E0B0E0EBEBD6
:10357000FAE10C94032DEE24E394F12C00E213E025
:103580009E012F5F3F4F42E153E064E083E00E94E1
:103590000B13C82E882339F100E080E01DC0D090C5
:1035A0003F03D00E2D2D30E0A901435A5C4F7A0124
:1035B000E1E0F0E0EC0FFD1FE00FF11D1081FA01DA
:1035C0009081191BB12E1B149CF0912F17FD90E0D8
:1035D000191B111118C00F5F90913E030917F8F2E3
:1035E00081110E94550C8C2D2196E9E00C941F2D21
:1035F000BA94F70180818F5F808360E08D2D0E94F7
:103600009C1A8C2DE0CF1F5FF70180818150808351
:1036100061E08D2D0E949C1A8C2DDBCFA5E0B0E0DF
:10362000E4E1FBE10C94002D7C01FC018381948199
:10363000892B31F08081918189238F3F09F0EBC381
:103640002596ECE00C941C2D0E948F0C182F682FEF
:1036500089819A810E94030D69817A81812F0E945C
:10366000180B8C01FC01E851FC47E730F10588F5A7
:10367000EC52F24D0C94512D26E241EE61EEC70161
:103680000E943D1A8091ED028770D1F2F70182818C
:103690008823B1F280914B0382FFD2CF82E00E9457
:1036A000500DCECF27E245EE65EEE9CF26E241EEA2
:1036B00060EEE5CF27E245EE64EEE1CF26E241EE93
:1036C00062EEDDCF27E245EE66EED9CF28E241E09B
:1036D000EBCFF7018281882309F4C4C310926F04F1
:1036E000C8019057839708F0A7C384E090E00E9438
:1036F0008E2D90934B0380934A03F801E150F047DD
:10370000E232F10520F4E552F24D0C94512D8091F6
:103710004A03816080934A0395C080914B0388607F
:1037200080934B038FC080914A038260F3CF8091D6
:103730004A038460EFCF80914A038860EBCF809189
:103740004B038160EDCF80914B038260E9CF809184
:103750004A038061DFCF80914A038062DBCF809192
:103760004A038064D7CF0E94821580914A03806803
:10377000D1CF80914A038C60CDCF80914B03836081
:10378000CFCF80914A038E7FC5CF80914B03877F37
:10379000C7CF80914A038D7FBDCF80914A038B7F35
:1037A000B9CF80914A03877FB5CF80914B038E7F3D
:1037B000B7CF80914B038D7FB3CF80914A038F7E2B
:1037C000A9CF80914A038F7DA5CF80914A038F7B3B
:1037D000A1CF0E94821580914A038F779BCF809161
:1037E0004A03837F97CF80914B038C7F99CF809141
:1037F0004A0382FB992790F921E0922790FB82F9F6
:1038000090FB83F987CF80914B03982F909591700F
:103810008E7F892B90FB81F983CF90914A03892F6A
:103820008F7B96FF806476CF0E94821590914A0329
:10383000892F97FB87F980586DCF61E08EE090E08B
:103840000E94A42D60914A0370914B0384E090E0A4
:103850000E94C22D0E94821515CF60E0EFCF90919B
:103860004A03892F8F7E94FF806154CF90914A0341
:10387000892F8E7F90FF81604DCF90914B03892FD0
:10388000877F93FF88604CCF85E3F5C280917104F8
:1038900091E08927809371041092620180917004F5
:1038A000816080937004EECE41EB59E06BEB79E0E0
:1038B0000E943209E7CE4BEB59E061EB79E0F8CF9B
:1038C0004DE959E067EA79E0F3CF47EA59E06DE95D
:1038D00079E0EECF43E859E060E979E0E9CF40E9EB
:1038E00059E063E879E0E4CF49E659E066E779E03A
:1038F000DFCF46E759E069E679E0DACF4DE459E0F9
:103900006BE579E0D5CF4BE559E06DE479E0D0CFB8
:1039100081E00E94ED06B6CE0E948215FFEF24E3FF
:103920003CE0F15020403040E1F700C000000E9430
:103930007F0F6FEF7FEF90E080E00E94C22D0E942A
:103940009E1880914B0382FB882780F991E089279C
:103950000E94D811F701828100811181882309F426
:1039600049C0C8010E948F0CD82E682FC8010E9440
:10397000030DB8018D2D0E94180B0E94370B8C018E
:10398000882EF701A280958092943FE09322809147
:10399000ED028770F1F0CA2CAA20E1F0812F807F20
:1039A000803451F080E2800F883098F0911004C08C
:1039B000812F807E803269F080914B0382FF09C0A5
:1039C00082E00E94500D8091ED028770CC24C39458
:1039D0008111C12CB12EB2942FE0B222FBE0FB1575
:1039E00008F474C0EB2DF0E0E350F24D0C94512D2F
:1039F00080E0AECFC8010E94D00CD82EBACF212FC4
:103A00002F70D22E107F19F0D29490EFD922AA20D5
:103A1000B9F0DD2069F080E2800F883010F081106D
:103A200009C080916703D82AD09267030E94670E6D
:103A3000802F4AC08091F602D82AD092F602F6CFA3
:103A4000802F0E948C19DD2009F440C0005E0830F0
:103A500010F0811004C08D2D0E945E0C06C0D09421
:103A60008091F602D822D092F6020E94670E2EC0F4
:103A7000312F3F70D32E107F103219F0D29480EF87
:103A8000D822882089F081E0881609F47CC0AA2019
:103A900009F486C0992009F47CC0F701858180FF74
:103AA000C7CF8F70858375C020914B0322FD43C023
:103AB000AA20D9F1DD2039F080916703D82AD0926D
:103AC00067030E94670E80E00E94C919EB2DE85041
:103AD000FF0B349710F40E942010CC20A9F08091A5
:103AE000ED0280FD11C0F7011282859585958595BF
:103AF0000E946C0DC7010E940E1B8091ED028595FE
:103B0000859585950E943E0D85E0F701DE011196B1
:103B100001900D928A95E1F709811A81C8010E94EE
:103B2000D00CB8010E94180B8BCD80E00E948C193C
:103B3000DD2061F290CFAA20A1F0909168038D2D35
:103B4000892B911003C00E94AB0EC0CFE1E09E1202
:103B5000FACF22FFBBCF891709F4B8CF809368034F
:103B6000B5CF911006C00E94580C8D2D0E94A40E56
:103B7000ADCFF1E09F1609F4A9CF8D2D0E94A40EC0
:103B80000E94580CA3CFAA2031F025E0291508F493
:103B90009DCF8D2DD8CF34E0391508F497CFE5CFE0
:103BA000992019F3F9E38F122FC12FEF37EE83E03D
:103BB000215030408040E1F700C0000025C1812F36
:103BC00086958695837061F0813009F07FCFC801BA
:103BD0009370A11002C080E090E00E94920876CF1E
:103BE000C8019370A11002C080E090E00E94B70865
:103BF0006DCF6A2D802F0E94B41868CF812F8370FB
:103C000009F03FC0A11062CF402F42954695477002
:103C1000440F440F802F8F7090E0042E02C0880F55
:103C2000991F0A94E2F730E020E004FF09C02FE07A
:103C300030E002C0220F331F4A95E2F720953095FD
:103C4000169516951370123099F078F44091F7029A
:103C50005091F802113039F0822B932B8423952355
:103C60000E947C0D33CF842B952B822B932BF8CF86
:103C7000822B932B2091F7023091F8028227932711
:103C8000EFCF8695AA2011F0812F8170882309F447
:103C90001DCF402F429546954770440F440F802F0B
:103CA0008F7090E0042E02C0880F991F0A94E2F7EB
:103CB00030E020E004FF09C02FE030E002C0220F16
:103CC000331F4A95E2F72095309516951695137097
:103CD000123099F078F440916503509166031130E9
:103CE00039F0822B932B842395230E94390DEECE3D
:103CF000842B952B822B932BF8CF822B932B209107
:103D000065033091660382279327EFCF1F70AA20A7
:103D100029F0812F0E946C0D802F15CF802F0E94DB
:103D2000A40E812F0E943E0DD1CE802F92EF8916D6
:103D300099F1981570F0E0EF8E16D1F0F1EF8F1633
:103D400091F0AA2009F45BC0911072CE812F8F717F
:103D500027C023EF821639F134EF8312F2CF80911E
:103D60004B0382FD2EC0812F8F71AA20D9F218C07B
:103D7000AA2069F084E0891508F4A8CE1F7181E0BB
:103D800090E002C0880F991F1A95E2F7B8CF95E02E
:103D9000991508F49BCEF2CF812F8F71A110C2CF5D
:103DA0000E946C0D93CE90E080E0AA2009F49DCF94
:103DB0001F7181E090E002C0880F991F1A95E2F709
:103DC00094CFAA2089F01F71812F0E946C0D8091E1
:103DD0004B0382FF07C0E8E01E9FC00111248360EF
:103DE0008093ED02812FDCCF81E00E94500DF1E045
:103DF000F91508F06BCE82E00E94500D67CE992035
:103E000039F0893309F4D1CE802F0E948C195ECE0F
:103E1000812F8F7187CF85E0DE01119601900D9281
:103E20008A95E1F7F701228189819A8121110CCCD1
:103E30000E94D00C182F10CC0631FCE71F0749F563
:103E4000809167038A7A91E009F490E090939C0254
:103E500069E2811165E384E992E00E9478080E949A
:103E6000670E10CC06312CE7120799F580919C0261
:103E700081110ACD89E2E6E9F2E02CE932E0919184
:103E8000891303C0DF0111971C922E173F07B9F762
:103E9000E6CF03303CE7130709F44BCD50F401158E
:103EA0009CE7190709F438CD01301C4709F447CDC8
:103EB00051CD0B35FCE71F0709F49ACD0C352CE7E3
:103EC000120709F43ECD0A351C4709F043CD81E0C5
:103ED0003FCD809167038272F801E052F847E531E7
:103EE000F10508F037CDE75FF14D0C94512D1F938C
:103EF000CF93DF938091BA02807F09F04BC080910D
:103F0000B702882309F446C08091EC02C091BB023D
:103F10004091B5025091B6026091B8027091B90219
:103F2000D42FD52316E0C817A9F190E061157105CB
:103F3000A9F1DF3F99F1189FF001199FF00D1124AD
:103F4000DF01A454BD4F11962C911197251326C063
:103F50002C91241323C012962C91129721111EC06C
:103F600013962D913C91261B370B283C3105B0F45C
:103F70008091BA028F7080618093BA02EF53FD4F37
:103F800080818F708061808385EB92E00E940E1BA0
:103F90000E94850CDF91CF911F9108950196877043
:103FA000C2CFA1E1B0E0E7EDFFE10C94002D8C0160
:103FB00085E0F801DE011D9601900D928A95E1F7EA
:103FC000F801E28085EB882E82E0982E4091B802BD
:103FD0005091B9024115510509F430C19091B502D3
:103FE0002091B602892F82238F3F09F427C1D08008
:103FF000C180A380B480F090B702B501641B750B3B
:10400000FF2009F4E7C08091BA02382F307F683C66
:10401000710508F0ABC0311178C0FE2C2C1114C012
:104020009D1112C0E11010C08F7080618093BA02A0
:10403000C4010E940E1B8091BA02F80185838F2D66
:104040006196ECE00C941C2DA114B104C9F18D2DE6
:104050008C218F3FA9F181E08E2580FF05C04E2D78
:104060006C2D8D2D0E94650CA114B10459F18D2D7C
:104070008C218F3F39F181E08E25F82FF170BF2E12
:1040800080FF39C04E2D6C2D8D2D0E94650CA82E01
:10409000811131C0DD86CE868D859E850E94C30C40
:1040A000292F22952F70243078F49F702230A8F0A9
:1040B0009923B9F0F8019581907F99F4FA2CBFCF3C
:1040C00080E0CBCF80E0D9CF2A5F2F70223068F01C
:1040D000C8010E940E1BAB2CF1CF992311F088234D
:1040E00069F3805E883050F3F3CF803F38F3815F0F
:1040F000833070F7E3CFEE2009F4A1CF8091BA02AC
:1041000081608093BA02F12C9ACF2C1105C09D11C9
:1041100003C0EE2009F477C0C8010E94810D8823F6
:1041200009F1EE20F9F08091BA02803270F020910E
:10413000B5023091B60238872F831986BB86AA86CE
:104140008C87CE0107960E940E1B86E0F801A5EB36
:10415000B2E001900D928A95E1F70E94771FFF244B
:10416000F3946DCFC8010E940E1BF9CF31110AC024
:1041700085EB92E00E940E1B86E0F40111928A9575
:10418000E9F7C1CF2C110EC09D110CC0E1100AC07F
:104190008583C8010E940E1B86E0F40111928A9566
:1041A000E9F74DCFC8010E94810D8823D9F2EE2096
:1041B000C9F28091BA02803240F22091B50230916A
:1041C000B6023A8329831B82BD82AC828E83CE01E4
:1041D0000196B9CF683C7105F8F6FE2CEE2011F27D
:1041E0002C111EC09D111CC08091BA0280FD0FC011
:1041F000982F907F61F08583903F31F0982F907FCA
:10420000905F8F70892B8583C8010E940E1B86E00A
:10421000F801A5EBB2E001900D928A95E1F70FCF7E
:10422000C8010E94810D811190CF8091BA028160F6
:104230008093BA02C8010E940E1B01CFEE2009F440
:1042400091CFC8010E94810DF82E882309F48ACFEE
:1042500086E0F801A5EBB2E001900D928A95E1F7B6
:104260008091B5029091B6020E94C30C0E94771F04
:10427000E6CEA7E1B0E0EFE3F1E20C94092D4B8B21
:104280005C8B6D8B7E8B8F8B61111092F6021A8A7C
:10429000198A85E0FE017396DE011D9601900D924C
:1042A0008A95E1F786E0FE013D96DE0117960190C2
:1042B0000D928A95E1F7CE0107960E94D11F8111D8
:1042C00012C086E0FE013796DE01119601900D9234
:1042D0008A95E1F78A859B85892B29F088859F81BE
:1042E00089238F3F81F516E08091EC029091BB020B
:1042F000891317C06796E3E00C94252D96E0929FF2
:10430000D001939FB00D1124A454BD4FFE013196EE
:1043100001900D929A95E1F78093BB020E94850C63
:10432000E2CF819FC001112484549D4F0E94D11F70
:10433000882301F38091EC0290E001968770992721
:104340008093EC02D1CF2091BB0230E0C9010196ED
:10435000877099274091EC024817190679F60E9458
:1043600082151092BB021092EC0286E0E5EBF2E0BF
:10437000DF011D928A95E9F7B6CFACE0B0E0E3EC3F
:10438000F1E20C94FF2C8E010F5F1F4F88E0D801E3
:104390001D928A95E9F786E4C82E81E0D82EF12C8B
:1043A000E12CAA24A394B12C26E4822E21E0922EA3
:1043B000F60181916F018F3F09F442C0F894E82F14
:1043C000E295EF70F0E021A18F70A50102C0440FCB
:1043D000551F8A95E2F7CA01922F982B91A392A1BB
:1043E0008095892382A3789400C0E0E4F1E0712CE9
:1043F00031E021912F3F09F46BC0A22FA295AF703D
:10440000B0E090968C9190E02F7002C095958795C2
:104410002A95E2F780FD5CC0832F782A330F8E1631
:104420009F0639F7F601319780818F3F11F00E9486
:104430001C0A50EA5A95F1F7F801EE0DFF1D708243
:104440008FEFE81AF80AA4E0EA16F10409F0B0CFF9
:1044500048E050E0B80180E493E00E94602D0097AE
:1044600041F028E0F801A0E4B3E001900D922A9514
:10447000E1F700914903892B69F181E08093FD0206
:104480000E944F159093FC028093FB028091FB02E7
:104490009091FC020E944015059700F110E0045B2A
:1044A0001C4F44E050E060E473E0C8010E94602DBE
:1044B000B12C892B51F084E0E0E4F3E0D8010190C5
:1044C0000D928A95E1F7BB24B3941092FD0207C0C8
:1044D00080E0A3CF8091FD028111D8CFB12C0E9442
:1044E000FD0FA82EE0914903882309F49FC0198687
:1044F0001A861B861C860E2F10E0045B1C4F8091D1
:1045000039038A3008F05CC040EB53E1BE01675FBD
:104510007F4FC8010E94CA0F882309F476C04FEE6E
:1045200052E1BE01675F7F4FC8010E94CA0F882316
:1045300009F46BC045EB5AE1BE01675F7F4FC801CC
:104540000E94CA0F882309F460C04FEE51E1BE01FA
:10455000675F7F4FC8010E94CA0F882309F455C0C6
:1045600045EC52E1BE01675F7F4FC8010E94CA0F50
:10457000882309F44AC046EA52E1BE01675F7F4FD3
:10458000C8010E94CA0F882309F43FC01092390362
:104590008091480390E044E050E0BE01675F7F4FA8
:1045A000845B9C4F0E94602D21E020930403892BA3
:1045B000F1F4A12C8A2D8B292C96EDE00C941B2D67
:1045C0008091FE029091FF020E944015843F91402D
:1045D00008F09ACF80910403882359F3FE0139969D
:1045E00084E0DF011D928A95E9F710920403E091BF
:1045F0004803F0E0E45BFC4F89859A85AB85BC8578
:1046000080839183A283B383D5CF809139038F3F79
:1046100031F08F5F809339038A3008F4B9CF0E945C
:104620004F159093FF028093FE02D4CF0091480370
:1046300010E0045B1C4FF0E0E45BFC4F84E0A7E17A
:10464000B3E001900D928A95E1F764E070E087E1B4
:1046500093E00E941C098093160384E0EBE1F3E0F1
:10466000D80101900D928A95E1F74091620350E0E4
:104670006091610370E0635A7C4FCE0109960E94FD
:104680006D2D89858093200361E070E0CE0109964D
:104690000E941C0980931F03C0902103D090220325
:1046A000E0902303F0902403809100039091010394
:1046B000A0910203B0910303C816D906EA06FB06CF
:1046C000D1F0C0920003D0920103E0920203F09275
:1046D00003030E94FD0F81110EC00E946C08C61AD0
:1046E000D70AE80AF90AC0923A03D0923B03E09253
:1046F0003C03F0923D0386E0E5E2F3E0A1E7B4E09D
:1047000001900D928A95E1F780912C03882319F08E
:104710000E94FA0E4FCF0E94DF0E4CCFA5E0B0E012
:10472000E4E9F3E20C94082D0E944F158C0180916E
:10473000F9029091FA0280179107A1F08FEF898317
:104740008A831B820E944F158160782F9D838C8302
:1047500049815A816B818D810E9439211093FA021F
:104760000093F9022596E4E00C94242D1F921FB6C5
:104770001F9211248F939F93AF93BF938091510405
:10478000811113C08091520490915304A09154045C
:10479000B09155044196A11DB11D80935204909390
:1047A0005304A0935404B0935504BF91AF919F91CB
:1047B0008F911F901FBE1F901895CDB7DEB72D9714
:1047C0000FB6F894DEBF0FBECDBF85B7806885BF3A
:1047D00085B7806885BF84B7877F84BF0FB6F8949C
:1047E000A8958091600088618093600010926000BD
:1047F0000FBE80E890E00FB6F8948093610090932C
:1048000061000FBE8AE19AE0909393028093920236
:104810000E940F070E94B0078091E200846080939D
:10482000E2007894809163048823A1F01091E9005C
:104830001F709091EC00892F817090FD80E8182BFB
:104840001092E9008091E80083FD0E94A9151F7075
:104850001093E90082E084BD93E095BD9AEF97BD87
:1048600080936E0010923A0310923B0310923C0327
:1048700010923D0384988C988FE891E00197F1F7AE
:1048800000C000008FB18295817080934A010E9420
:10489000FD0F81110E94842B90914A0181E098279D
:1048A00090936103A82FA91BA0933F0390914A0105
:1048B0008093620390914A0180933E0380914A0164
:1048C000811106C086EF8093540187EF80935301D6
:1048D00020915401E22FE295EF70F0E061A12F707A
:1048E00081E090E0AC0101C0440F2A95EAF7342F33
:1048F0003095362331A322A1242B22A320915301EA
:10490000E22FE295EF70F0E031A12F7001C0880F27
:104910002A95EAF7982F9095932391A392A1892B3A
:1049200082A38FE891E00197F1F700C00000109199
:10493000620363E673E044E551E083E5E82E81E03D
:10494000F82EFB0128C0DA012D91AD01822F82954E
:104950008F7090E0DC0190968C9190E02F7002C0F7
:10496000959587952A95E2F78170D7019D917D01F4
:10497000292F22952F7030E0D90190962C9130E0AC
:104980009F7002C0359527959A95E2F790E020FD3B
:1049900092E0892B81938E2F861B8117A0F2809144
:1049A0004A01811120C081E38093460183E3809313
:1049B000470182E38093480186E38093490186E0C2
:1049C000E6E6F1E0DE01119601900D928A95E1F79D
:1049D000FE013196A0E4B1E0CE01079621912D931E
:1049E0008E179F07D9F780914A0194E0811190E0DA
:1049F0009093490384E0891B8093480306E411E007
:104A0000EAE4EE2EE1E0FE2EF80181918F018F3F66
:104A100011F00E941C0AE016F106B1F700E411E063
:104A2000D8018D918D018F3F11F00E941C0AB1E0D9
:104A300006341B07A9F788E0ECE4F3E0DF01282F38
:104A40001D922A95E9F7E0E4F3E0DF011D928A95D3
:104A5000E9F790E080E00E948E2D873E9E4F11F096
:104A60000E94E41382E090E00E94862D809354031C
:104A700084E090E00E948E2D90934B0380934A0334
:104A80000E94BD21EFEFF6E721E0E150F040204029
:104A9000E1F700C000000E94BD217C990FC0E4E056
:104AA000F0E0E45BFC4F808185FF0AC06FEF7FEF91
:104AB00090E080E00E94C22D0E947F0FE0E0F0CFE6
:104AC00083E090E00E94862D90E00E947C0D90E0B3
:104AD00080E00E948E2D873E9E4F21F00E94E413BD
:104AE0000E94BD1181E08093700446E050E06CE1CB
:104AF00070E081E794E00E94762D1092700480911E
:104B000071048C7F11F40E94BD1183E080938903AE
:104B100080E2809377040E943E2A6DE070E08FE986
:104B200092E00E94B50E892BE9F58091890363E03C
:104B300070E081FD9AC08CE992E00E94B50E892B4D
:104B400089F56DE070E08CE892E00E94B50E892B4B
:104B500049F50E946C08605A75418F4F9F4F6093D2
:104B60004504709346048093470490934804EAE711
:104B7000F4E080E092E0DF019C011D922150304082
:104B8000E1F7F0938106E09380068FEF9FEF90931B
:104B900079048093780481E080934A0480934904E7
:104BA00010928A030E94FD0F811102C00E94872B80
:104BB0008BE491E090934E0480934D0470E4672E53
:104BC0008091630400E112E1853009F48CC00E94F9
:104BD000BD2155E5E52E53E0F52E6CE4C62E63E0CD
:104BE000D62ED601F70191918D9123E0ED35F20794
:104BF00009F483C09817B9F30E94FD0F882E10E0C6
:104C0000D6010D916D01F70191907F01901629F168
:104C1000B12CAA24A3949026892D8A21B1F0882052
:104C2000A1F0BF82188791E08A2D802309F490E0DB
:104C300099870E944F158160782F9B878A874F81C3
:104C4000588569858B850E943921B394AA0CF6E0BA
:104C5000BF12E2CFF701319700831F5F183081F652
:104C60000E946C08EE24E3944DC089E992E065CF80
:104C700080916304843039F10E944B100E94DF0E52
:104C80001092510488E190E00FB6F894A8958093B3
:104C900060000FBE6092600083B7817F846083BF35
:104CA00083B7816083BF7894889583B78E7F83BFF5
:104CB0000FB6F894A8958091600088618093600099
:104CC000109260000FBE80916204882361F00E9400
:104CD000BD21ECE4F3E081918111B0C3A4E5B3E020
:104CE000AE17BF07C1F780916304853009F4C0CFC8
:104CF0000E9482150E9420106ACF98137DCF0E94D7
:104D00008E23E12C0E94FD0F0E944B10C12CF12C30
:104D100080916203C81608F483C0F1100E94550CFC
:104D200080914A04882309F4ACC180918B0390914F
:104D30008C030E944015C29708F483C10E944F154E
:104D400090938C0380938B038AE794E09093810681
:104D5000809380060E94FD0F882309F479C260E8E1
:104D600070E08CEA92E00E94DC0880917704F4E025
:104D70008F9FC0011124811522E0920714F090E06A
:104D800080E086589B4F90938106809380068CE24A
:104D900093E00E94590E82E793E00E94590E8091A1
:104DA000650390916603009709F4C1C081FFB8C004
:104DB00082E693E00E94590E82E793E00E94590E2A
:104DC0001091680380916703182B012F08781474E1
:104DD000002309F4B2C08BE993E00E94590E84E9E4
:104DE00093E0112309F4B1C086E993E00E94590EC3
:104DF0008DE893E0111102C08AE893E00E94590EF9
:104E0000002309F4A8C087E893E00E94590E82E8C5
:104E100093E00E94590E1111A8C088E793E0A7C043
:104E20000C2D10E0F801EC5AFE4F8081E82FE2953E
:104E3000EF70F0E0E0A1F0E08F7002C0F595E7952B
:104E40008A95E2F7E170D801AD5ABE4F2C91A22F9E
:104E5000A295AF70B0E090968C9190E02F7002C058
:104E6000959587952A95E2F780FD52C080E08E2BBC
:104E7000D801AD59BC4FEC919E2F9370891709F45E
:104E800045C0EE0FEE0FE82BEC93D0906103DC0CE5
:104E9000EF70F0E0E955FE4F015A1C4F8081D801B8
:104EA0009C91890F8C93B12C843084F0ED2DF0E02F
:104EB000E35AFC4F80818F5F80830E94FD0FB82EE4
:104EC000882341F160E08D2D0E949C1AF8018081B9
:104ED0008D3F84F4ED2DF0E0E35AFC4F808181504A
:104EE00080830E94FD0FB82E8823B9F061E08D2DDC
:104EF0000E949C1AD8018C91082E000C990B64E03A
:104F000070E00E943D2DF8018083FB28C39400CF00
:104F100082E0ADCFBB24B394D9CFBB24B394EACF06
:104F200082FF03C082E593E045CF80FF03C082E4A7
:104F300093E040CF82E393E03DCF88E993E00E9485
:104F4000590E111105C080E993E00E94590E54CF0B
:104F500082E993E04BCF84E893E00E94590E11233D
:104F600089F180E893E00E94590E8BE793E00E945C
:104F7000590E1091680380916703182B012F01715E
:104F80001272002321F181EC93E00E94590E8AEB0A
:104F900093E0112321F18CEB93E00E94590E83EBF7
:104FA00093E00E94590E002311F18DEA93E00E94D4
:104FB000590E88EA93E00E94590E111123C08EE920
:104FC00093E022C08EE793E00E94590E26CF8EEB2D
:104FD00093E00E94590E111107C086EB93E00E94E6
:104FE000590E80EB93E0DDCF88EB93E0D6CF8AEAD1
:104FF00093E00E94590E112309F425C186EA93E03B
:105000000E94590E81EA93E00E94590E0E942010DE
:10501000182F80ED93E010FF02C083ED93E00E9413
:10502000590E8AEC93E011FF02C08DEC93E00E94D0
:10503000590E84EC93E012FF02C087EC93E00E94CB
:10504000590E8091780490917904892B09F007C159
:10505000809149048823A9F00E946C0800914504BE
:10506000109146042091470430914804601B710B55
:10507000820B930B6F3F7F4F8F4F9F4710F40E941F
:10508000DF0EE11001C0F1100E94FA0E86E0E5E9A2
:10509000F3E0DE01119601900D928A95E1F71092EE
:1050A0009703109298031092990310929A038B81A0
:1050B0009C81892B09F44AC08091930390919403B9
:1050C0000E9440159C0190918E03992309F4D1C14F
:1050D00025313105D8F19F3F19F09F5F90938E03E2
:1050E0001B81112359F00E94FA099FEF11160CF44D
:1050F00091E0899F802D1124809397031C811123B7
:1051000059F00E94FA099FEF11160CF491E0899F63
:10511000802D112480939803309197033323B1F0AD
:1051200020919803222391F045EB3403C001112410
:10513000992309F473C19093970345EB24039001DD
:105140001124332309F46EC1309398038D819E811D
:10515000892B09F44AC080919103909192030E9497
:1051600040159C0190918F03992309F47DC121354D
:105170003105D8F19F3F19F09F5F90938F031D81F8
:10518000112359F00E94D8099FEF11160CF491E0F9
:10519000899F802D1124809399031E81112359F03A
:1051A0000E94D8099FEF11160CF491E0899F802D81
:1051B000112480939A03309199033323B1F0209105
:1051C0009A03222391F045EB3403C0011124992363
:1051D00009F42CC19093990345EB24039001112409
:1051E000332309F427C130939A0346E050E0BE010F
:1051F0006F5F7F4F85E993E00E94602D892B61F4FA
:105200008091970390919803892B90919903892B12
:1052100090919A03892B11F00E945B1586E0FE01A4
:105220003196A5E9B3E001900D928A95E1F70E94CD
:10523000201090918D03891709F4C2CC80938D03BF
:105240000E946C08BDCC84EA93E00E94590EB7CE50
:1052500060E072E086ED93E00E94DC08F2CE80917F
:105260004A04882309F4F4CE80918A038111F0CE98
:105270000E94FA0E209178043091790421153105AD
:1052800009F4E6CE80E041E050E0082F10E02A016A
:10529000082E02C0440C551C0A94E2F7B2016223A6
:1052A0007323672B11F48F5FF0CF9091890390FFE8
:1052B0009CC0880F880F880F8093570110925A0165
:1052C000895F8093580183E080935B0124E630E09E
:1052D00047E050E065E571E088E70E94DE2A892B0F
:1052E00009F0B6CEA80125E0440F551F2A95E1F735
:1052F0008091890380FF8BC0E9E6F3E080E2DF0163
:105300001D928A95E9F7EBEBF1E0FD87EC8707EB5F
:1053100011E097E0A92E99249394AC85BD852D9139
:10532000BD87AC87F80121908F01240E352E311CEA
:10533000C10186589B4F1C01E22FF0E0E759FC4F5A
:1053400030E020E07A2C721AB92C022E01C0BB0C7E
:105350000A94EAF7610190E0D6018D916D018B21ED
:10536000672D691B6770862E062E000C770BB82FF1
:1053700001C0BB0F8A94EAF78B2E71956195710974
:105380006770772701C086956A95EAF7882A808139
:10539000882A80829F5F9830F9F62F5F3F4F3196C1
:1053A0002830310579F6EFEBF1E02C853D85E217E9
:1053B000F30709F0B2CF04E610E020E230E049E65E
:1053C00053E060E488E70E94FF2A892B09F040CE71
:1053D0004094509480917804909179044822592205
:1053E000509279044092780433CE8295880F80766B
:1053F00080935701980136952795369527952093E8
:105400005A01815E8093580110925B015FCF46582C
:105410005B4F04E610E020E230E0D3CF81E08093E0
:1054200097038BCE81E08093980390CE81E08093A8
:105430009903D2CE81E080939A03D7CE09BD19BDDE
:1054400009B400FEFDCF8091D8008F7D8093D800F5
:105450008091E00082608093E0008091E00081FD17
:10546000FCCF0E9482153FCC2B30310508F084CE52
:10547000BCCE2B30310508F030CE68CE1092B9008A
:105480008CE08093B8000895B0E0A0E0EAE4FAE28E
:105490000C94012DB82EEB010E944F156C01EE24E7
:1054A000E394F12CC431D10560F025E0E22EF12C1B
:1054B000CF3FDC0731F0CE0164E170E00E94E62CC2
:1054C0007B0184EAA82E94E8992E1092BC00A09249
:1054D000BC000E944F158C018091BC0087FF0DC05D
:1054E0008091B900887F8830F9F08091B900887F79
:1054F0008031D1F00FEF1FEF08C0C8010E944015A6
:10550000E816F90648F70EEF1FEFCF3FDC07E9F288
:10551000C6010E944015C817D907B8F6C801CDB713
:10552000DEB7EBE00C941D2DB092BB009092BC0056
:105530000E944F158C018091BC0087FF0AC08091AA
:10554000B900887F883111F08034A1F610E000E0C6
:10555000E5CFC8010E944015E816F90660F7D3CFE1
:105560000F931F93CF93DF93EB018093BB0084E8ED
:105570008093BC000E944F158C018091BC0087FF76
:1055800011C02091B900287F81E090E0283211F409
:1055900090E080E0919581959109DF91CF911F91E5
:1055A0000F910895CF3FDC0741F3C8010E944015D9
:1055B000C817D90710F78EEF9FEFEFCFB0E0A0E04C
:1055C000E4EEFAE20C94042D6B018A017901B90131
:1055D0000E94442AE6010C0D1D1DC017D10711F0D1
:1055E00097FF08C024E92093BC00CDB7DEB7E8E000
:1055F0000C94202DB70189910E94B02AEECFB0E023
:10560000A0E0E5E0FBE20C94042DC62F6A017901CD
:10561000B8010E94442A97FD0CC0B8018C2F0E944B
:10562000B02AE601EC0CFD1CCE15DF0511F097FF4A
:1056300008C024E92093BC00CDB7DEB7E8E00C94A5
:10564000202DB80189910E94B02AEECF84E9809381
:10565000BC0008958EE14A9B02C08150E1F74A9B4D
:10566000FECF08955A9880E28A95F1F75A9A0895E4
:10567000FC013BE03A95F1F798E020E080E031E072
:1056800040E14A95F1F7880F4A9B02C081602327C9
:1056900042E04A95F1F7000040E14A95F1F7915058
:1056A00079F790E19A95F1F799B132E03A95F1F7EF
:1056B000000040E14A95F1F792FB992790F9922773
:1056C0002081920F90830895A1E0B0E0EAE6FBE22A
:1056D0000C94062D19828C017C01E60EF11C0E152E
:1056E0001F0541F481E09981911180E02196E6E067
:1056F0000C94222D0E942A2BCE0101960E94382B59
:10570000F80181938F01EBCF529A5A9A08955298DB
:105710005A9AEA9AE9E6F0E080818F7C80830895C6
:105720006150770B91E001C0990F6A95EAF720E08C
:1057300031E0911108C0222391F05A9A80E28A95B3
:10574000F1F75A980895492F482339F05A9A232798
:1057500040E24A95F1F79695ECCF5A98F9CF5A98CE
:10576000EDCFFF920F931F93CF93DF93EC018C014A
:10577000060F111DC017D10729F4CDB7DEB7E5E03C
:105780000C94232DF9900E94322B68E08F2D0E94FB
:10579000902BF0CF1F920F920FB60F9211240F9300
:1057A0001F932F933F934F935F936F937F938F93A9
:1057B0009F93AF93BF93EF93FF93CF93DF930F929A
:1057C000CDB7DEB719820E942A2BCE0101960E9426
:1057D000382B082F069506950695282F22952570BB
:1057E000902F9570290F922F937026952695920FE2
:1057F000982797708981982B09F05CC0093008F0D0
:1058000059C080E18A95F1F75A9A529A82E08A95B6
:10581000F1F700C05A9888E0089F80011124D80150
:10582000A050BF4F1696ED91FC9117973097A9F0B5
:105830006091A5017091A60114962D913C91159748
:10584000260F371F11968D919C911297680F791F23
:1058500013964C9113978C910995F801E050FF4FE6
:105860006381662351F02091A5013091A6018481C6
:105870009581820F931F0E94B12B0E94322B80E1F1
:105880008A95F1F75A9852985A9A80E18A95F1F7D9
:10589000F801E050FF4F6081662351F02091A5018F
:1058A0003091A60181819281820F931F0E94642B07
:1058B0000E942A2B0F90DF91CF91FF91EF91BF9122
:1058C000AF919F918F917F916F915F914F913F9198
:1058D0002F911F910F910F900FBE0F901F90189551
:1058E0000F931F93CF93DF93EC0109970CF04CC0FB
:1058F000F894529A5A9885E08A95F1F700009C2F07
:10590000969595708C2F8570980F892F837096953A
:10591000969523E0CC0FDD1F2A95E1F7980F8E01B5
:10592000092B0E94322B00C068E0802F0E94902B30
:1059300080E18A95F1F752985A9A4A9B1EC087E0F7
:1059400090E04A991CC0FE01E050FF4F638166233E
:10595000F9F02091A5013091A60184819581820FF3
:10596000931F0E94642B811113C0529A5A9A789403
:10597000DF91CF911F910F91089500C0DECF019765
:1059800029F4529A5A9A789480E0F2CF00C0D9CF85
:105990000E942A2B80E28A95F1F75A98529A80E168
:1059A0008A95F1F7C050DF4F6881662351F020914E
:1059B000A5013091A60189819A81820F931F0E94CF
:1059C000B12B0E94322B789481E0D2CFAA1BBB1B53
:1059D00051E107C0AA1FBB1FA617B70710F0A61BEF
:1059E000B70B881F991F5A95A9F780959095BC0110
:1059F000CD0108952F923F924F925F926F927F92C6
:105A00008F929F92AF92BF92CF92DF92EF92FF92CE
:105A10000F931F93CF93DF93CDB7DEB7CA1BDB0B7A
:105A20000FB6F894DEBF0FBECDBF09942A8839881F
:105A300048885F846E847D848C849B84AA84B98426
:105A4000C884DF80EE80FD800C811B81AA81B98132
:105A5000CE0FD11D0FB6F894DEBF0FBECDBFED0146
:105A60000895991B79E004C0991F961708F0961BBA
:105A7000881F7A95C9F78095089597FB072E16F42D
:105A8000009407D077FD09D00E94E62C07FC05D0D2
:105A90003EF4909581959F4F0895709561957F4F45
:105AA0000895EE0FFF1F0590F491E02D0994FB017E
:105AB000DC0102C005900D9241505040D8F7089586
:105AC000FB01DC0104C08D910190801921F441504B
:105AD0005040C8F7881B990B0895FB01DC0102C0F8
:105AE00001900D9241505040D8F70895DC01CB0150
:105AF000FC01F999FECF06C0F2BDE1BDF89A3196DE
:105B000000B40D9241505040B8F70895F999FECF76
:105B100092BD81BDF89A992780B50895A8E1B0E0BB
:105B200042E050E00C94782DDC01A40FB51F4150E9
:105B3000504048F0CB01840F951F2E910E94A52D57
:105B400041505040D0F70895262FF999FECF92BDCD
:105B500081BDF89A019700B4021639F01FBA20BD32
:105B60000FB6F894FA9AF99A0FBE08950396272F64
:105B70000E94A52D0E94A42D252F0E94A52D242F23
:105B80000C94A52D0196272F0E94A52D0C94A42DD1
:105B9000F894FFCF8816B0164818B0164818E316C8
:105BA0000417481801180E18561B5A1B3C1B521B91
:105BB0005E1B621B661BC11B361CC91B931B971BFC
:105BC000CD1B9B1BD11BDD1BA71B2F1CAB1BE11B84
:105BD000AF1BE51B0D1CB31BE91B141CB91BEF1BF2
:105BE000F71B9F1BD51BA31BD91BBD1BF31B031C42
:105BF0001D1C2D1C8D1BC51B3D1CFF1CFF1C381DB7
:105C0000381DDF1DF91D661D661DFE1D861E951EB5
:105C1000951E461C541C5B1C601C651C6A1C6F1C7A
:105C2000741C791C7E1C831C881C421B421B421B5B
:0C5C3000421B421B421B421B421B421B3A
:105C3C000000000100000000000000040100000052
:105C4C000405000000000000000000010900000035
:105C5C00000000010A000000040B0000000000001E
:105C6C00070F0000000000000116000000000000FB
:105C7C0032363331F7F697C634350169086B0F6449
:105C8C000F5D0F66940021007F220003FFFF00FFD1
:105C9C0000010300FF80946697C63435818283E24D
:105CAC0000E900EA00B500B600B700CD008301CCD6
:105CBC00008A01920194012102230224022502266A
:105CCC000227022A02B300B4006F0070009F01CBC0
:105CDC00019F02A002160300FF0100010000FFFF5C
:105CEC000000010001FF000008101818100800182F
:105CFC001716151413191211100F0E1A0D0C0B0A7E
:105D0C0009080706FFFFFF333231302F2E342D2CBC
:105D1C002B2A29352827262524232221FFFFFF5D46
:105D2C00113B0319071D31463368375F3F503A3C2E
:105D3C00375527442532232125102A551544133273
:105D4C000D211410185504440232002103100700D1
:105D5C0007001800298311A503C707C3319A3378AC
:105D6C0037813F903AA4378B279C25AE23BF25D093
:105D7C002A8B159C13AE0DBF14D0188B049C02AE4D
:105D8C0000BF03D007E007E018E02902020202027C
:105D9C0002040404040404040404040404040404B9
:105DAC0004040404040402020202020204040404B3
:105DBC000404040404040404040404040404040497
:025DCC000400D1
:00000001FF
